:1000000005280000000000000229123086000030A0
:100010008500831688308100093086000030850015
:1000200083128C018B100B160B118B168B17061677
:10003000D820980006121808733A031928201808C7
:10004000713A031933201808633A03193720172827
:100050006320C220013A031930286F30D0200800F5
:100060007230D0200800B5206F30D0200800D82092
:10007000F6209F009F0ED820F6209F04D820F6205F
:100080009900990ED820F6209904D820F6209A00DD
:100090009A0ED820F6209A047F20013A031953289B
:1000A0006F30D02056287230D02056281D0EEB20FD
:1000B000D0201D08EB20D0201E0EEB20D0201E08E3
:1000C000EB20D0200800DD20023085008611831649
:1000D00086118312FF30E7200F309600083085002C
:1000E0003030E720023085003030E720960B6E2854
:1000F00083168615831204308500E3200800DD2076
:1001000019089B001A089C00C220013A0319B32861
:100110001030960086198A280330E720000000007E
:10012000861183169B1F861183129C0D9B0D033035
:10013000E7200000000000009E0D9D0D1E10861996
:100140001E140000000000000000000000008316E4
:1001500086158312861DAA28960B8A289F0B7F2856
:10016000B128E3200034E3200134DD200230850093
:10017000C2203030E72000308500831686158312B8
:10018000E320080020309600861DC4281430970014
:10019000861DCD28970BC8280034960BC42801343F
:1001A0000C18D02893000A30920094000C14080018
:1001B0000C1DD82815080C1108000C080339031D64
:1001C000DD288B1308000B118B108B170800FF3EE6
:1001D000031DE72808000F39A000F63E0318F32896
:1001E0002008303E08002008573E0800A000B03E1E
:1001F0000318FE282008D03E0F3908002008A93E29
:100200000F3908008D0003088E0083120B1D0F2983
:10021000CE3081000B110C1832218C1821210B1AC1
:1002200017218D0E0E0883000D0E8B1708008B1CF6
:100230000800093091000B128B108C1401308F00D4
:1002400008008F0B080002308F00900C90130618E6
:100250009017910B08008C108B100B16100895004E
:100260000C150800940B08000230940012080A3A9A
:10027000031D3D2986109203080013188614131CD1
:0E02800086100314930C920B08000C1008005B
:00000001FF
